:020000040000FA
:0E0000000219FDD2D3A68A08C2D3320211F62D
:0300130002054E95
:0F001B00302F0AD2D3B285868B08C2D33281D759
:10002B0075C800203E0653E6DF020436752741856E
:09003B0055CC8556CD43E6203278
:03005B0002055C3F
:10006300302454C521C59B30E61620181002043BEA
:1000730053917FC050C05122759B808136C5213278
:10008300C52120180132759100856C94856D957595
:1000930050FE202410C56EF552047553FE6003759F
:1000A300500014C56E75910443E680C21832203E99
:1000B30004D0E0012B8045759B80C0E0E59B65275C
:1000C30020E63120182B103821C2CA10CFE0E5CC2E
:1000D300F4F5CCE5CDF4F5CD303E0FC0D0C3E5CC7F
:1000E3009555E5CD95564012D0D0B23ED2CAD0E058
:1000F30032D0E032D0E020188D32D0D08555CC8577
:1001030056CD80E6D0E075C80053E6DF813604069D
:10011300080C10182030406080A0C00000000000D0
:1001230000000000000000000000000000000000CC
:1001330000000000000000000000000000000000BC
:1001430000000000000000000000000000000000AC
:10015300000000000000000000000000000000009C
:10016300000000000000000000000000000000008C
:10017300000000000000000000000000000000007C
:10018300000000000000000000000000000000006C
:10019300000000000000000000000000000000005C
:1001A300000000000000000000000000000000004C
:1001B300000000000000000000000000000000003C
:1001C300000000000000000000000000000000002C
:1001D300000000000000000000000000000000001C
:1001E300000000000000000000000000000000000C
:1001F30000000000000000000000000000C55204E1
:1002030004700714C5528553503214C55232D2A01C
:10021300C2AFC292D29475D53CD2AF759F30754FA1
:10022300266169D2A0C2AF75D533D2AF759F23754E
:100233004F376169D2A0C2AFC294D29075D533D281
:10024300AF759F31754F4C6169D2A0C2AF75D50FA1
:10025300D2AF759F03754F5D6169D2A0C2AFC290E3
:10026300D29275D50FD2AF759F32754F726169D235
:10027300A0C2AF75D53CD2AF759F13754F11D21A7B
:100283006169D2A0C2AFC294D29275D53CD2AF7588
:100293009F31754F9A6169D2A0C2AF75D50FD2AFA6
:1002A300759F23754FAB6169D2A0C2AFC292D29042
:1002B30075D50FD2AF759F30754FC06169D2A0C29B
:1002C300AF75D533D2AF759F13754FD16169D2A086
:1002D300C2AFC290D29475D533D2AF759F32754FEA
:1002E300E66169D2A0C2AF75D53CD2AF759F0375E5
:1002F3004F85D21A61693024068045D2198136753B
:100303009100856994856A957550FE202410C56B0C
:10031300F552047553FE600375500014C56B759157
:100323000443E680C219C218202002D2187527415F
:10033300759BB075C8008555CC8556CD43E62032F4
:10034300C2AF759100856994856A95759104D2AFA2
:100353007550FE43E680C219D21875218075274176
:1003630043E620020063302426C0D0C2AF7591005B
:10037300C5942563C594C5953564C595759104D217
:10038300AF5003439180D0D07550F943E680327566
:1003930091008563948564957550F9202410C56593
:1003A300F552047553F9600375500014C5657591D2
:1003B3000443E6803253E6DF75C800C2A07591009E
:1003C300856694856795854F50202410C568F5523E
:1003D30004854F53600375500014C5687591044339
:1003E300E680C0E0C0D0E55C64036038D21BE8C59A
:1003F30057F8C3E5F9A660F56096F608E5FAA66135
:10040300F56120DF0D96F608E54DA662F56296F6D6
:10041300807420E7F096F608E54D0480ED20E7119F
:100423000562806C85F960E5FAF561854D6220DF30
:10043300EC805D20240761B8C521759B80C2AF7530
:100443009100856694856795759104D2AF854F5069
:1004530043E68053E6DF75C800C2A0C0E0C0D0E524
:100463005C640360BFD21BE8C557F8C3E5F9A66017
:10047300F56096F608854D62E5FA20DF20A661F562
:100483006196F6087600E8040444F0C557F8055C65
:10049300E5245403600E2021020532801D20E7DD90
:1004A300056280D9A218922730190F20230C201837
:1004B30009B193D226D0D0D0E032C3E55B95354065
:1004C30009C291C293C29575D53FD0D0D0E053E60F
:1004D300DFC21932C2A8C0D0C0E0C28ED22D758A45
:1004E30000E508B4B72E30332DD22FD28543A42094
:1004F3007508B9758921538EF0758B9785748C8532
:10050300738AC28DC28FD2BBD28CD28E43A80AD03B
:10051300E0D0D032D22E85718B7508A7D2A8D2AA8B
:10052300D0E0D0D032E54E2418F54EE52260021516
:1005330022C3E5396005753A00A149E53A2401F57E
:100543003A5003753AFFD0D0D0E032C2AA85718BFE
:10055300D28E85F94A85FA4B32C0E0E5F730E619C9
:1005630053F7DFE5F9E5FA30E10F853BE9853CEA2E
:10057300853DFB853EFC53F7BF10DF03D0E032C25D
:10058300DF054DC0D0E54E954D609AD0D0D0E03216
:10059300C2AF75910075C800759B00D2AFC2AFC2E0
:1005A30091C293C295C290C292C29475D53FD2AF05
:1005B300227901801879038014790A8010790F80D9
:1005C3000C791E80087964800479C8800075A913AA
:1005D30075A71075C10075A700781474F0000000AA
:1005E300D5E0FAD8F6D9F275A71075C13075A70012
:1005F30075A903227901801479038010790A800C8C
:10060300791E80087964800479C88000759100752B
:10061300949875954075910453E67FE9C0E01208FC
:100623000CD0E0F9E59130E7F2D9E12278FF202000
:100633002879A1E76023E559601F74C48559F084C4
:100643008536F030210375F005A4F8C5F060027813
:10065300FFC3E895425002A842884122C3E55D9456
:10066300A0E55E9400E5415003148001046002F5A7
:1006730041220543C3E5439408404F30EDF47543ED
:100683000079A0E76043E5BE7006E5446019800D7C
:10069300C3E5BD9544600EE5445005600A14800728
:1006A3000460FA8002E544F544C39548401B754055
:1006B300C0C394044013754080C39404400B754039
:1006C30040C39404400375400022E54024105002C7
:1006D30074FFF54022743279A687F0A4C5F0A2F71F
:1006E30033F54222755D00755EF0227A1C7B3C80F7
:1006F300127A147B4B800C7A107B5A80067A0A7B21
:10070300788000EFD5E0012275A91375A71075C194
:100713000075A7007902E4C292D5E0FDD293D5E03B
:10072300FDC293D5E0FDD292D5E0FDE920E002D2EF
:100733009130E002D295EFD5E0FDE920E002C291CD
:1007430030E002C2957496D5E0FDD9CAEAF8D5E047
:10075300FDD8FBDBAEC29275A71075C13075A7003B
:1007630075A90322788676090876017892760308BC
:100773007628087650087604087602087607087605
:1007830001087600087600227888E6C39403D23203
:100793005002C232C230E630E102D230A23092318E
:1007A3007886E6149001119378A6F67886E6F536F6
:1007B300C394025003753602789CE67535FFB40284
:1007C300037535A0B4030375358278A0E6F8600697
:1007D30074282409D8FCF5482278A5E6F95403D2F5
:1007E300B07002C2B0E9540CD2B17002C2B1E95484
:1007F30030D2B27002C2B2E954C0D2B37002C2B3F3
:1008030022120BEF2212122922102DF5A22BB03344
:10081300B02F40F12275460075470012059375808D
:10082300FF75F12075A4007580FF75D4FF7590C026
:1008330075F23F75A53F7590C075D53F75A00075DE
:10084300A60175A72075CC0175A700E5B525E06065
:100853000975A71075CF0075A70075E34075E2020F
:100863001205931207671213CC754C017557F07577
:1008730058F075510275A71075C13075A70075A999
:1008830003C2AF1205CC789886071206EE1205C094
:100893001205C01205C01206F41205C01205C012DB
:1008A30005C01206FA1205C01205C01205C01207D0
:1008B300001207001205C81207DC22C2AF53A4DFDF
:1008C300D28575A91375A71075C10075A700754664
:1008D30000754700AAE475E4D578FA79FA308509FA
:1008E300D9FBD8F7021C008AE422C2AF12078B128D
:1008F300059375A71075C13075A70075A903C225A7
:1009030075D84075D90975F781759E03759601757C
:10091300DB4275DA4275A82175E61043B801759B71
:1009230080759D3075D10C75BCB975BB1075E880A9
:1009330075B2017534001205B42230580675E45DB2
:10094300D22B2275E4D5C22B22C2AF78988607A298
:100953002B4007120700120700221206FA1206FAAA
:1009630022D2AF12060B120607C3E53994014002E7
:1009730080EFC2AFA22B78988607402CC0071206DF
:10098300EED2AF120607C2AFD0071206EEC007D2EF
:10099300AF120607C2AFD0071206EEC007D2AF12DE
:1009A3000607C2AFD007800912070012070012071B
:1009B30000C289D2AF12060B22E4F55DF55EF55F46
:1009C300F530F5317520000520300145752000050F
:1009D30030E530F4703B0531789AE67819146012EB
:1009E300783214600D787D14600878FA146003750A
:1009F3003100C3E5319840191205931205B415313E
:100A030075300078998607C2AF120700D2AF12067D
:100A1300071205FFE5227002C3221205F73028A74B
:100A2300C3E5399401500AC3E56F9401501E0209CE
:100A3300CA120607E5227002C322756F00757000A3
:100A4300D3227546A57547F112140622AF6F12140F
:100A53009F754600754700C22880BFC2AF7557F027
:100A63007558F0755C00D2AF120593E4F543F52396
:100A7300F524F55B7543081205F775E89030EDFD35
:100A8300A8BDE5BE7001F8884412067575430812C7
:100A930006D8854240854241303207C230302902B0
:100AA300D230D220753200E4C2AF85F96085FA6195
:100AB300854D62D2AFF55DF55E755F0875595012CD
:100AC30010461211CE20300812029A1202858006B7
:100AD30012022612021175E890102613101B121031
:100AE3002D1EA22BB033B02F4011101A1880EA61CB
:100AF300BDD1761210461211CE80DE12122980D992
:100B0300120BEF80D420240312062F302403120685
:100B13005F12067530202785424079187A0CC3E5A9
:100B23003299400EC220D2218A3385424085424108
:100B3300800CC3E53994014003020AD961C5302111
:100B43001F20231CE533147006C221D2228087F5AF
:100B530033203207C3E53994014003020AD9806286
:100B630075340020320F78FA79A4E760027803C362
:100B7300E53A98504DE52260493032152030052082
:100B83002907800D3029028008202305D2238542BE
:100B93004078F03023058542407819C3E5599850D1
:100BA30003020AD930231BC223C230302902D230B8
:100BB300D22175331285424041D90534E5396002AB
:100BC30061C8753400120593752400C289120607A3
:100BD30012059375230078A4E66006D290D292D2D0
:100BE30094C3E53494044002C322D322102E0CE4B0
:100BF300AE72FCFBFA790878A78002A1AFE6FDC3C9
:100C03009CC39E40F69EEB33FB08E6FCC39DC39E4C
:100C130040E99EEB33FB08E6FDC39CC39E40DC9E8C
:100C2300EB33FB08E6FCC39DC39E40CF9EEB33FB37
:100C330008E6FDC39CC39E40C29EEB33FB08E6FC63
:100C4300C39DC39E40B59EEB33FB08E6FDC39CC327
:100C53009E40A89EEB33FB08E6FCC39DC39E409BCE
:100C63009EEB33FB088002A1AFE6FDC39CC39E400D
:100C7300F69EEA33FA08E6FCC39DC39E40E99EEA6A
:100C830033FA08E6FDC39CC39E40DC9EEA33FA08B0
:100C9300E6FCC39DC39E40CF9EEA33FA08E6FDC33C
:100CA3009CC39E40C29EEA33FA08E6FCC39DC39EE2
:100CB30040B59EEA33FA08E6FDC39CC39E40A89E56
:100CC300EA33FA08E6FCC39DC39E409B9EEA33FACF
:100CD30008EBC46B6A54F0F9EAC4302B01F454F006
:100CE300C3996002A1AFEBF4C454F0F9EAF4C4541D
:100CF3000F49FAEBF4C4540FFBC3EAF99460FAEB1F
:100D03009400FB5020C3E97B007A0079006016C38E
:100D1300135006F9C3956F600AE9F56F7570007992
:100D23000080020570303227C3EA94D0F8EB9407B1
:100D3300F9400BE8FAE9FB202909D229800530297B
:100D430002C229203102B229C3EA33FAEB33FBEBA7
:100D53002B3B3BF9C3EB13FBEA13FAEA29FAEB3417
:100D630000FB30E3047AFF7BFFE5245403601B2080
:100D73002218E54233F9EB7007C3E99A4002E9FA16
:100D8300E534C4332AFAEB3400FBC3EA33C4540F0B
:100D9300F8EB33C454F048F87005EA60027801E5D3
:100DA3007960021579802475220A80140579E57922
:100DB30070021579C3E5799432500280EA753900DF
:100DC300202F07D2AAD2A87508A7228839D228E8EB
:100DD3006003753A00C3E540FC95414002AC41C352
:100DE300EC95395008EC75F008A4FAABF0EBF4136A
:100DF3001392D5A2E75401F9EAF4FC13A2D513F830
:100E0300E54C23F54CEC5403243783554C600BE835
:100E13002401E9340020E10208F9C3E89405FAE962
:100E23009400FB50047A007B00883B893C8A3D8B0D
:100E33003E75220A53F7DF43F740202F0343E610A2
:100E4300A1C300115577C3EC13FCEB13FBEA13FAB0
:100E5300860508860608860708084300F08858C3F5
:100E6300EF941840027F18C3ED33FDEE33FEEF33EA
:100E7300FFE161A858302479AA5DAB5EC3EAC4548C
:100E83000FFCEBC4FD54F04CCA9AFAED540FCB9B04
:100E9300FBE60303543FFC08E60303FD54C04C2A5E
:100EA300FAED543F3BFB0808084300F0D55CCDC284
:100EB3001B88587C008C5F8B5E8A5DECC40354F8FE
:100EC300F9EBC403540749F5597800302702780138
:100ED300E55B75F007A4F9E5F028F5F0E9A2F01356
:100EE300A2F113A2F213F8C3947850027878885BC6
:100EF30022AA5DAB5EAC5F302003020E49E559C305
:100F03009403400A94045003020FC1020F88ECC4F7
:100F1300F9540FFFE954F0FEEBC4F9540F4EFEE908
:100F230054F0FDEAC4540F4DFDC3EA9DFAEB9EFB5A
:100F3300EC9FFC860508860608860708084300F030
:100F43008858EF0303F9543FFFE954C0CE0303F974
:100F5300543F4EFEE954C0CD0303543F4DFDEA2DEB
:100F6300FAEB3EFBEC3FFC8C5F8B5E8A5DD55C133A
:100F7300C21BECC3941840097C18E4F55DF55E8C44
:100F83005FC1BEC176EC0303F9543FFFE954C0FED1
:100F9300EB0303F9543F4EFEE954C0FDEA03035447
:100FA3003F4DFDC3EA9DFAEB9EFBEC9FFC860508D3
:100FB300860608860708084300F0885880A0ECC41A
:100FC30023F9541FFFE954E0FEEBC423F9541F4EE9
:100FD300FEE954E0FDEAC423541F4DFDC3EA9DFA24
:100FE300EB9EFBEC9FFC860508860608860708082F
:100FF3004300F08858C3EF13FFEE13FEED13FD0219
:101003000F61C3E55D2323F954FCFAE95403FBE5BF
:101013005E2323F954FC4BFBE95403FCE55F2323D4
:1010230054FC4CFCC3E49AFAE49BFBE49CFC240CC4
:101033004005E47CF4FAFBC2AF8A6C8B6D8C6ED2F4
:10104300AF801AE559C394024004C22480B4D22469
:10105300C2AF756C98756D40756EFFD2AF302005C9
:101063007F030210847892E6FFC3E55B948240110C
:101073000FC3E55B94A040010FC3EF940640027FCA
:1010830005E55FC4FC540FFAEC54F0F9E55EC4FCCB
:10109300540F49F9EC54F0F8E55DC4540F48F8C314
:1010A300E89440FBE99400FCEA9400FD400CC3EB98
:1010B3009401EC9400ED940050057B01E4FCFD20C9
:1010C3002047C3E49BF8E49CF9E49DFAE8FBE9FCC0
:1010D300EAFDD3ED13FDEC13FCEB13FBC2AF886900
:1010E300896A8A6BD2AFC3EF94037065C2AF886617
:1010F30089678A68D2AF28F8EC39F9ED3AFAC2AFBA
:10110300886389648A65D2AF22E4C2AFF569F56A60
:10111300756BECD2AFC2AFF56CF56D756EECD2AFFB
:10112300C3E5329401500FC2AF7563007564E07577
:1011330065FFD2AF800DC2AF7563007564F075654E
:10114300FFD2AFC2AF7566B07567FF7568FFD2AFE8
:101153002220E111EB28F8EC39F9ED3AFAC3EF94C8
:10116300034016803DE828F8E939F9EA3AFA74FFB2
:10117300FBFCFDC3EF94035029C2AF886689678ADD
:1011830068D2AFD3E56B13FAE56A13F9E569132B5C
:10119300FBE93CF9EA3DFAC2AF886389648A65D208
:1011A300AF22C2AF8B668C678D68D2AFD3E56B136A
:1011B300FDE56A13FCE5691328F8EC39F9ED3AFA11
:1011C300C2AF886389648A65D2AF22302401227A50
:1011D300007BFDE5590303543FF994034005E4FA0A
:1011E300C399FBD3EB13FBEA13FAC2AF8A558B56B1
:1011F300D2AF22C23353A4DFD2855388A5758C00A6
:1012030075892A85788E7508A785718BC2A9C2BB9B
:10121300D2AAD2A8D28CC22F32FBEA13FA0C8031A5
:1012230074FFFBFA8029E55FAB5EAA5DC403F85443
:1012330007FCE854F8CBC403F854074BFBE854F815
:10124300CAC40354074AFAEA24FFEB34FF50D1E43B
:10125300FCC3EB1370C3EC234B540FC4FBEAC4FA77
:10126300540F4BFBEA54F0FA6BC46B540F4A640FF0
:10127300FA78B974ADC0E07412C0E079757D13EAF1
:10128300540F242A83C0E0C005EAC4540F241F83EB
:10129300C0E0C005EB540F241583C0E0C005EBC4C8
:1012A300540F240A83C0E0C005227600D233220003
:1012B3000C1B24303F4B5766727C8693A2AFBC0055
:1012C300000000000000000000000000000000001B
:1012D300000000000000000000000000000000000B
:1012E30000000000000000000000000000000000FB
:1012F30000000000000000000000000000E7F60806
:10130300A67508A67708797522E7F608A67508A6D4
:101313007608A67508797522E7F608A67708797620
:1013230022E7F608A67708A67508797522E7F60876
:10133300A67508A67508A67608797522E7F608A6A5
:101343007608A67608797522E7F608A67608A675C4
:1013530008797622E7F608A67608A67508A6750822
:10136300797522E7F608A67508A676087976220924
:10137300E7F608A6770879752209E7F608A676083E
:1013830079762209E7F608A67608A6750879752204
:10139300E7F608A67508A67508A6750879762209E2
:1013A300E7F608A67508A6760879752209E7F60810
:1013B300A67508A6750879762209E7F608A67508C2
:1013C300A67508A67508797522901A0D78209132B2
:1013D300E520B4550AA39132E520B4AA0261F5755C
:1013E30046A57547F11207679106754600754700D4
:1013F3008105901A0378807B269132A308DBFA904B
:101403001A2922C2AF91759152901A007403913731
:10141300A374009137A374219137901A0378807BCA
:10142300269136A308DBFA91889166901A2922E463
:1014330093F622E6438F01538FFDFFC3E583941C8C
:10144300400122EF8546B78547B7F0538FFE22430D
:101453008F02438F018546B78547B7901A0DF05326
:101463008FFC22901A0D74559137901A0E74AA911D
:1014730037227A3079807820901A409132E520F330
:1014830009A3DAF7227A307980901A40E391370979
:10149300A3DAF9227C051205CCDCFB22EFC3940707
:1014A300400FEFD3940E5009E570C394065002C366
:1014B30022EF14B40E0040030215599014CC75F0BA
:1014C30003A4C58325F0C583730214F60214F60240
:1014D30014F60214F60214F6021559021503021546
:1014E3001002151D0215280215590215560215334F
:1014F30002153DEF24FEFF7899E6FD12164F805644
:101503007F033032027F017888A60780407F043052
:1015130032027F027888A607802D30323978881608
:1015230016C232803120322E78880606D2328026C7
:101533007888E630E002800F8013901A0BE49364FE
:10154300017888F630E006D230D2318009C230C249
:10155300318003120A45E4F56FF570D322E4F58870
:10156300780876A7C228F56FF570C2A975892AF5A0
:101573008DF58CC2AFD2AAD2AB757856758E5675DF
:101583008851C2AF7571E2757214C2AFD258120995
:101593003D7573C17574FE7575FC7576F77577F1D6
:1015A30075790AD2AF120607E579C3940A5001226E
:1015B300C2AFC25812093D75790AD2AF120607E5C8
:1015C30079C3940A5001227571C3757228C2AFD2D0
:1015D3005812093D7573FC7574FD7575F67576EBD8
:1015E3007577E075790AD2AF120607E579C3940AD5
:1015F300500122C2AFC25812093D75790AD2AF1207
:101603000607E579C3940A500122C3227F08758136
:10161300CD43FF807597DE7597AD75EF06E4F5A9A9
:10162300F5A9AE070FA806E4F6EF70F61208181234
:1016330008BE1208ED12156050F512094C12096428
:101643001209BC50EA120A5E40F680E38F088D0946
:10165300C2AF120593E50814601414601814601CDB
:101663001460192404701AAF091206EE8013AF092F
:101673001206F4800CAF091206FA8005AF091207AF
:0616830000D2AF020607D1
:1019FD0002160F030021FFFFFFFFFFFF09FF01FF8D
:101A0D0055AA01FFFFFFFFFF03FFFFFF25D0285061
:0D1A1D0004FF02FF7AFF0701FFFF0000FF3A
:101A400023535F485F303523202020202020202092
:101A500023424C48454C492445464D3842323123B7
:101A60002020202020202020202020202020202076
:101C0000C2AFC2D37597DE7597AD7581C075A90057
:101C100075A90043FF80752438752503B1DE752949
:101C2000A5752AF143F12053A4DFD28575D4FF7541
:101C3000E3407DFA780379E67C1075220075230075
:101C4000901DEB7B06752498752501308502814B2C
:101C5000208508D8FBD9F9DCF781BD308508D8FB91
:101C6000D9F9DCF781BDB19EE493A3C39A6004DD8A
:101C7000C381BDDBDBB190600281347B08E493FA61
:101C8000A3B171DBF87A30B171752200752300B110
:101C900090EAFCEBFDC3ED94FE400EB1908A278BD9
:101CA00028ED30E0048A828B83B1907AC270D8C369
:101CB000ED94FE601950CEBD0029EC600F75200038
:101CC0007521FF752900752A000200008100A827F0
:101CD000A9280809D804D90281E0B194EAF281D494
:101CE0000D81A9C3ED94035051EDA2E092007AC595
:101CF000C3E5829400E583941C508C200010438F30
:101D000002438F018529B7852AB7F0300027A8271D
:101D1000A9280809438F01538FFDD804D902A135A2
:101D2000C3E583941C4003A3A11AE28529B7852A41
:101D3000B7F0A3A11A538FFC81857AC1BD030CE4CF
:101D400093A3FAB155DCF8B14D81858187AA22AB06
:101D500023B171EBFAEA6222752608C3E52313F575
:101D600023E52213F52250066323A0632201D52622
:101D7000EAB1DEB1DE75260AEAF4200102D285302E
:101D80000102C285B1DEC3134002C201D526EB2297
:101D9000B194EAFB208502A194308502A1997526B1
:101DA00008AE24AF25C3EF13FFEE13FEB1E2B1DEA0
:101DB000C3EA133085024480FA30E703632201C38B
:101DC000E52313F523E52213F52250066323A063D0
:101DD0002201D526D9E52265236523F52222AE24EA
:101DE000AF250E0FDEFEDFFCD20122424C48656CAF
:091DF0006934373164E8B20601E0
:00000001FF
